:020000040000FA
:020000000528D1
:080008003028031383160030B9
:100010008500013086000030870000308800003005
:10002000890083128316FF309F00831200309F00E7
:100030008117011381120116811501158114011414
:100040008B170B178B120B168B110B118B100B10C0
:10005000FF30850086008700880089006400630007
:100060008B106400FF30CA00FF30CB000130C600A7
:10007000FF30C1000A30CA00CA0B3C28061C4628C3
:10008000CB0B3A28C60AC61B28283828FF30CC00DC
:100090004D08FF30CE00FF30CF003C27E130CE00CE
:1000A000FF30CF003C27C030CE00FF30CF003C27D0
:1000B0008030CE007F30CF003C270030CE003F3074
:1000C000CF003C270030CE003F30CF003C2700302F
:1000D000CE003F30CF003C270030CE001F30CF0095
:1000E0003C271230CE001F30CF003C273330CE00EB
:1000F0001F30CF003C273330CE001F30CF003C27CD
:100100003330CE001F30CF003C273330CE001F30BD
:10011000CF003C273330CE001F30CF003C27333098
:10012000CE001F30CF003C273230CE001F30CF0032
:100130003C273030CE001F30CF003C273030CE007F
:100140003F30CF003C273030CE003F30CF003C273F
:100150003030CE003F30CF003C27B030CE007F3073
:10016000CF003C27B030CE00FF30CF003C27F1302D
:10017000CE00FF30CF003C27FF30CE00FF30CF0055
:100180003C27FF30CE00FF30CF003C27FF30CE00B1
:10019000FF30CF003C27FF30CE00FF30CF003C27A0
:1001A0000030CE000030CF003C270030CE000030C1
:1001B000CF003C270030CE000030CF003C2700307D
:1001C000CE000030CF003C270030CE000030CF0002
:1001D0003C270030CE000030CF003C270030CE005E
:1001E0000030CF003C27FF30CE00FF30CF003C274F
:1001F000FF30CE00FF30CF003C27FF30CE00FF3075
:10020000CF003C27FF30CE00DF30CF003C27FF304F
:10021000CE001F30CF003C27FE30CE001F30CF0075
:100220003C27F830CE001F30CF003C27E030CE0016
:100230001F30CF003C27C030CE001F30CF003C27FE
:100240000030CE001F30CF003C270030CE001F30E2
:10025000CF003C270030CE007F30CF003C2703305A
:10026000CE00FF30CF003C270730CE00FF30CF005C
:100270003C270130CE00FF30CF003C270030CE00BD
:100280007F30CF003C270030CE001F30CF003C270E
:100290000030CE001F30CF003C27C030CE001F30D2
:1002A000CF003C27F030CE001F30CF003C27FC3081
:1002B000CE001F30CF003C27F030CE001F30CF00E3
:1002C0003C27E030CE001F30CF003C278030CE00EE
:1002D0001F30CF003C270030CE001F30CF003C271E
:1002E0000030CE007F30CF003C270130CE00FF3001
:1002F000CF003C270730CE00FF30CF003C27033033
:10030000CE00FF30CF003C270030CE00FF30CF00C2
:100310003C270030CE001F30CF003C270030CE00FD
:100320001F30CF003C27C030CE001F30CF003C270D
:10033000E030CE001F30CF003C27F830CE001F3019
:10034000CF003C27FE30CE001F30CF003C27FF30CF
:10035000CE001F30CF003C27FF30CE00DF30CF0073
:100360003C27E130CE00FF30CF003C27C030CE002C
:10037000FF30CF003C278030CE007F30CF003C27BD
:100380000030CE003F30CF003C270030CE003F3061
:10039000CF003C270030CE003F30CF003C2700305C
:1003A000CE001F30CF003C271230CE001F30CF00D0
:1003B0003C273330CE001F30CF003C273330CE00F7
:1003C0001F30CF003C273330CE001F30CF003C27FA
:1003D0003330CE001F30CF003C273330CE001F30EB
:1003E000CF003C273330CE001F30CF003C273230C7
:1003F000CE001F30CF003C273030CE001F30CF0062
:100400003C273030CE003F30CF003C273030CE008C
:100410003F30CF003C273030CE003F30CF003C276C
:10042000B030CE007F30CF003C27B030CE00FF3060
:10043000CF003C27F130CE00FF30CF003C27FF300B
:10044000CE00FF30CF003C27FF30CE00FF30CF0082
:100450003C27FF30CE00FF30CF003C27FF30CE00DE
:10046000FF30CF003C270030CE000030CF003C27CB
:100470000030CE000030CF003C270030CE000030EE
:10048000CF003C270030CE000030CF003C270030AA
:10049000CE000030CF003C270030CE000030CF002F
:1004A0003C278030CE000030CF003C271E30CE00ED
:1004B0003F30CF003C273F30CE003F30CF003C27BD
:1004C0003F30CE001F30CF003C273F30CE001F30E2
:1004D000CF003C273F30CE001F30CF003C273F30BD
:1004E000CE001F30CF003C271E30CE001F30CF0083
:1004F0003C270030CE001F30CF003C270030CE001C
:100500001F30CF003C270030CE003F30CF003C27CB
:100510000030CE003F30CF003C270030CE003F30CF
:10052000CF003C278030CE007F30CF003C27E13029
:10053000CE00FF30CF003C27FF30CE00FF30CF0091
:100540003C27FF30CE00FF30CF003C27FF30CE00ED
:10055000FF30CF003C27FF30CE00FF30CF003C27DC
:100560000F30CE00FF30CF003C270F30CE00FF30E1
:10057000CF003C270F30CE00FF30CF003C270F309C
:10058000CE00FF30CF003C270F30CE00FF30CF0031
:100590003C270F30CE00FF30CF003C270F30CE007D
:1005A000FF30CF003C27FF30CE00FF30CF003C278C
:1005B000FF30CE00FF30CF003C27FF30CE00FF30B1
:1005C000CF003C27FF30CE00FF30CF003C27E1308A
:1005D000CE00FF30CF003C27C030CE00FF30CF0030
:1005E0003C278030CE007F30CF003C270030CE004B
:1005F0003F30CF003C270030CE003F30CF003C27BB
:100600000030CE003F30CF003C270030CE001F30FE
:10061000CF003C271E30CE001F30CF003C271E30BD
:10062000CE001F30CF003C273F30CE001F30CF0020
:100630003C273F30CE001F30CF003C273F30CE005C
:100640001F30CF003C273F30CE001F30CF003C276B
:100650001F30CE001F30CF003C271E30CE001F3091
:10066000CF003C270C30CE001F30CF003C270C3091
:10067000CE001F30CF003C270C30CE003F30CF00E3
:100680003C270C30CE003F30CF003C279E30CE00C0
:100690003F30CF003C279E30CE007F30CF003C273C
:1006A000DE30CE00FF30CF003C27FF30CE00FF30E1
:1006B000CF003C27FF30CE00FF30CF003C27FF307B
:1006C000CE00FF30CF003C273F30CE001F30CF00A0
:1006D0003C271F30CE001F30CF003C270F30CE000C
:1006E0001F30CF003C270F30CE001F30CF003C27FB
:1006F0000730CE001F30CF003C270330CE001F3024
:10070000CF003C270130CE001F30CF003C27013006
:10071000CE001F30CF003C270030CE001F30CF006E
:100720003C270030CE001F30CF003C273030CE00B9
:100730001F30CF003C273030CE001F30CF003C2789
:100740003830CE001F30CF003C273C30CE001F3069
:10075000CF003C273E30CE001F30CF003C273E303C
:10076000CE001F30CF003C273F30CE001F30CF00DF
:100770003C273F30CE00FF30CF003C27FF30CE007B
:10078000FF30CF003C27FF30CE004F083F30CC0079
:10079000FF30CD003C273F30CC001F30CD003C2740
:1007A0003E30CC001F30CD003C273E30CC001F3007
:1007B000CD003C273C30CC001F30CD003C273830EA
:1007C000CC001F30CD003C273030CC001F30CD0096
:1007D0003C273030CC001F30CD003C270030CC000F
:1007E0001F30CD003C270030CC001F30CD003C270F
:1007F0000130CC001F30CD003C270130CC001F3031
:10080000CD003C270330CC001F30CD003C27073003
:10081000CC001F30CD003C270F30CC001F30CD0066
:100820003C270F30CC001F30CD003C271F30CC00C0
:100830001F30CD003C273F30CC001F30CD003C277F
:10084000FF30CC00FF30CD003C27FF30CC00FF3024
:10085000CD003C27FF30CC00FF30CD003C27DE3000
:10086000CC00FF30CD003C279E30CC007F30CD0047
:100870003C279E30CC003F30CD003C270C30CC00D4
:100880003F30CD003C270C30CC003F30CD003C2722
:100890000C30CC001F30CD003C270C30CC001F307A
:1008A000CD003C271E30CC001F30CD003C271F3030
:1008B000CC001F30CD003C273F30CC001F30CD0096
:1008C0003C273F30CC001F30CD003C273F30CC00D0
:1008D0001F30CD003C273F30CC001F30CD003C27DF
:1008E0001E30CC001F30CD003C271E30CC001F3006
:1008F000CD003C270030CC001F30CD003C2700301D
:10090000CC003F30CD003C270030CC003F30CD0044
:100910003C270030CC003F30CD003C278030CC005D
:100920007F30CD003C27C030CC00FF30CD003C27CD
:10093000E130CC00FF30CD003C27FF30CC00FF3051
:10094000CD003C27FF30CC00FF30CD003C27FF30EE
:10095000CC00FF30CD003C27FF30CC00FF30CD0075
:100960003C270F30CC00FF30CD003C270F30CC00AF
:10097000FF30CD003C270F30CC00FF30CD003C27AE
:100980000F30CC00FF30CD003C270F30CC00FF30C3
:10099000CD003C270F30CC00FF30CD003C270F307E
:1009A000CC00FF30CD003C27FF30CC00FF30CD0025
:1009B0003C27FF30CC00FF30CD003C27FF30CC007F
:1009C000FF30CD003C27FF30CC00FF30CD003C276E
:1009D000E130CC00FF30CD003C278030CC007F30B0
:1009E000CD003C270030CC003F30CD003C2700300C
:1009F000CC003F30CD003C270030CC003F30CD0054
:100A00003C270030CC001F30CD003C270030CC000C
:100A10001F30CD003C271E30CC001F30CD003C27BE
:100A20003F30CC001F30CD003C273F30CC001F3082
:100A3000CD003C273F30CC001F30CD003C273F305D
:100A4000CC001F30CD003C273F30CC003F30CD00E4
:100A50003C271E30CC003F30CD003C278030CC00FE
:100A60000030CD003C270030CC000030CD003C27CA
:100A70000030CC000030CD003C270030CC000030EE
:100A8000CD003C270030CC000030CD003C270030AA
:100A9000CC000030CD003C270030CC000030CD0031
:100AA0003C27FF30CC00FF30CD003C27FF30CC008E
:100AB000FF30CD003C27FF30CC00FF30CD003C277D
:100AC000FF30CC00FF30CD003C27F130CC00FF30B0
:100AD000CD003C27B030CC00FF30CD003C27B030FB
:100AE000CC007F30CD003C273030CC003F30CD00F3
:100AF0003C273030CC003F30CD003C273030CC009C
:100B00003F30CD003C273030CC001F30CD003C279B
:100B10003230CC001F30CD003C273330CC001F30AA
:100B2000CD003C273330CC001F30CD003C27333084
:100B3000CC001F30CD003C273330CC001F30CD001F
:100B40003C273330CC001F30CD003C273330CC0065
:100B50001F30CD003C271230CC001F30CD003C2789
:100B60000030CC001F30CD003C270030CC003F309F
:100B7000CD003C270030CC003F30CD003C2700307A
:100B8000CC003F30CD003C278030CC007F30CD0002
:100B90003C27C030CC00FF30CD003C27E130CC00FA
:100BA000FF30CD003C27FF30CC00DF30CD003C27AC
:100BB000FF30CC001F30CD003C27FE30CC001F3072
:100BC000CD003C27F830CC001F30CD003C27E03072
:100BD000CC001F30CD003C27C030CC001F30CD00F2
:100BE0003C270030CC001F30CD003C270030CC002B
:100BF0001F30CD003C270030CC00FF30CD003C271B
:100C00000330CC00FF30CD003C270730CC00FF3054
:100C1000CD003C270130CC00FF30CD003C27003018
:100C2000CC007F30CD003C270030CC001F30CD0001
:100C30003C278030CC001F30CD003C27E030CC007A
:100C40001F30CD003C27F030CC001F30CD003C27BA
:100C5000FC30CC001F30CD003C27F030CC001F30E2
:100C6000CD003C27C030CC001F30CD003C270030E9
:100C7000CC001F30CD003C270030CC001F30CD0011
:100C80003C270030CC007F30CD003C270130CC0029
:100C9000FF30CD003C270730CC00FF30CD003C2793
:100CA0000330CC00FF30CD003C270030CC007F303B
:100CB000CD003C270030CC001F30CD003C27003059
:100CC000CC001F30CD003C27C030CC001F30CD0001
:100CD0003C27E030CC001F30CD003C27F830CC0062
:100CE0001F30CD003C27FE30CC001F30CD003C270C
:100CF000FF30CC001F30CD003C27FF30CC00DF3070
:100D0000CD003C27FF30CC00FF30CD003C27FF302A
:100D1000CC00FF30CD003C27FF30CC00FF30CD00B1
:100D20003C270030CC000030CD003C270030CC0008
:100D30000030CD003C270030CC000030CD003C27F7
:100D40000030CC000030CD003C270030CC0000301B
:100D5000CD003C270030CC000030CD003C270030D7
:100D6000CC000030CD003C27FF30CC00FF30CD0060
:100D70003C27FF30CC00FF30CD003C27FF30CC00BB
:100D8000FF30CD003C27FF30CC00FF30CD003C27AA
:100D9000F130CC00FF30CD003C27B030CC00FF302C
:100DA000CD003C27B030CC007F30CD003C27303028
:100DB000CC003F30CD003C273030CC003F30CD0060
:100DC0003C273030CC003F30CD003C273030CC00C9
:100DD0001F30CD003C273230CC001F30CD003C27E7
:100DE0003330CC001F30CD003C273330CC001F30D7
:100DF000CD003C273330CC001F30CD003C273330B2
:100E0000CC001F30CD003C273330CC001F30CD004C
:100E10003C273330CC001F30CD003C271230CC00B3
:100E20001F30CD003C270030CC001F30CD003C27C8
:100E30000030CC003F30CD003C270030CC003F30AC
:100E4000CD003C270030CC003F30CD003C27803027
:100E5000CC007F30CD003C27C030CC00FF30CD002F
:100E60003C27E130CC00FF30CD003C27FF30CC00E8
:100E7000FF30CD003C2732284D1805144D1C0510BD
:100E8000CD188514CD1C85104D1905154D1D051166
:100E9000CD198515CD1D85114D1A05164D1E05124E
:100EA000CD1A8516CD1E85124D1B09144D1F091034
:100EB000CD1B8914CD1F89104C1809154C1C091124
:100EC000CC180714CC1C07104C1987144C1D871024
:100ED000CC198814CC1D88104C1A08144C1E08100C
:100EE000CC1A8715CC1E87114C1B07154C1F0711F8
:100EF000CC1B0816CC1F081264004F1886174F1C15
:100F00008613CF180617CF1C06134F1986164F1DD0
:100F10008612CF190616CF1D06124F1A86154F1EC0
:100F20008611CF1A0615CF1E06114F1B86144F1FB0
:100F30008610CF1B8817CF1F88134E1808174E1C1A
:100F40000813CE188816CE1C88124E1908154E1D8F
:100F50000811CE198815CE1D88114E1A07164E1E7F
:100F60000712CE1A8716CE1E87124E1B07174E1F6A
:100F70000713CE1B8717CE1F87134608C700000034
:100F80000000000000000000000000000000000061
:100F90000000000000000000000000000000000051
:100FA0000000C70BBF2F640008000A30C2001430D5
:100FB000C1006430C0006400C00BDC2FC10BD92F0E
:100FC000C20BD72F0800640008003C30C1000A3073
:100FD000C000C00BE92F6400C10BE72F64000800BC
:02400E00BF3FB2
:00000001FF
